:02000000E228F4
:1000060083160313851505158312261005190F2867
:0A001600261C0E280F2809280800F8
:10002000053084000008000883120313F0007011EB
:06003000700880000800CA
:10003600053084000008000883120313F000F01155
:06004600700880000800B4
:04004C0000000800A8
:100050001B208316851126202620051583122610C5
:1000600005193628261C3528362830282620262033
:1000700026202620262026202620262083168515A9
:06008000262026200800E6
:1000860083160313851526202620051526202620EF
:100096001B20831685112620262010208316051185
:0200A600080050
:1000A800013083120313B0008030B100B201003078
:1000B8003206031D612800303106031998282620CE
:1000C80026202620262010208316051126202620EB
:1000D800831231082F05F10000303205F20000309C
:1000E8007206031D79280030710603197E288316CD
:1000F800851581281B2083168511262026200515A5
:100108008312261005198C28261C8B288C288628F3
:100118003108F0003208F100F10CF00CF11370080E
:10012800B1007108B2005B28B001262026201020FB
:100138008316051126202620851526202620262010
:1001480026200515831226100519AE28261CAD2871
:10015800AE28A828B00126202620851DB4283014F2
:100168002620262026202620262026202620262057
:100178002620262026202620262026202620262047
:100188001020831605111B20831685118312300851
:04019800F00008006B
:10019C000730831203139F00FF3083168600810102
:1001AC0003208230FC00DD30FD00FD0BDB28FC0B56
:0801BC00DB2800000000080030
:1001C400CE2083120608A000A10100302106031DE1
:1001D400ED282A082006031953292008AA00A00D97
:1001E400A10D2010A00DA10D2010A00DA10D201017
:1001F400051E01298030A8002530A9000529E0301A
:10020400A8004730A900051F0A29AD01AE010E2937
:10021400FC30AD000E30AE0020082807F00029089D
:100224000318013E2107F1007008AB007108AC000F
:100234002D087007F30071080318013E2E07F4001F
:100244007308AB007408AC007308F0007408F10084
:10025400F10CF00CF113F10CF00CF113F10CF00CA7
:10026400F1137008A5007308A4004320C230831260
:10027400AF0054207008A7002508AF005420700870
:10028400A7002408AF0054207008A700CE30AF00A8
:1002940054207008A7009030AF0054207008A700C5
:1002A40028200230FC004B30FD00FD0B5729FC0BCD
:0602B4005729E3285C2934
:02400E006A2125
:00000001FF
